:040000008A11112828
:10000800FE00030EF1000408F2000A08F300831250
:1000180003137F08F4008A110A298A1161298312BF
:100028000313A4010830831603138E0007308312CC
:1000380003139F00831603138501063086003330AF
:1000480099000430980090308312031398006400DC
:100058008B01831603138C018C160B178B178312D5
:10006800031385018601A601A701A8013B28831275
:1000780003133008031D41287E282830F500750831
:10008800B200B0012D082C07F5002E087507F60000
:100098002B087607F7007708B1002F0831060319F7
:1000A800562857285B28A601A701A8017E28A90180
:1000B80003302902031C6128622864287E287E28D0
:1000C8002908013E2B3E840083130008803EF5007A
:1000D8002908263E8400750880000130F50075085F
:1000E800A90703302902031C7A287B2864287E2864
:1000F8007E287E280130B202B208031D8428852894
:100108008E282830F5007508B200B301A601A701B2
:10011800A8018E28A50103302502031C94289528E0
:100128009728B128B1282508263E84008313801F0C
:100138009E289F28A128A414A3282414A3280310C8
:10014800A40D0310A40D0130F5007508A5070330B0
:100158002502031CB028B1289728A301AA0103305F
:100168002A02031CB828B928BB28E428E4282A084E
:10017800263E8400831300086039F5002A08203ED3
:10018800840075088007031CCA28CB28D0280330B0
:10019800F5007508A304D528FC30F5007508A305FB
:1001A800D5280310A30D0310A30D0130F500750821
:1001B800AA0703302A02031CE228E328BB28E42804
:1001C8002308F5007508A4052408C039F50075084A
:1001D800A3000310A40D0310A40D0330F500750847
:1001E80086053F30F500750885052408F500750873
:1001F80086042308F500750885044230F500F50BE0
:10020800032964003B283B288A1111288C1E0D29DC
:100218000E295629502950291A08F00033082B3E78
:1002280084007008831380003308031D1C292129CA
:100238000130F0007008B3072129B308031D2529F0
:100248002629382933082B3E84000008AA3A031DC2
:100258002E292F2938290130F0007008B3072830DB
:10026800F0007008B200382905303302031C3D291C
:100278003E294329B301B0010314B00D4329181DC9
:10028800462947295029181233082B3E840080013B
:10029800B3011816502950298C1A532954291029AA
:1002A800562956297408FF0073088A0072088400CA
:1002B800710E8300FE0E7E0E0900AB01AC01AD018C
:1002C800AE01AF01B001B101B201B30183018A11DE
:0202D8001328E9
:02400E0010FFA1
:00000001FF
